:020000040000FA
:100000007D28820700340034003401340034003489
:1000100000340A34003400340034643400340034D2
:100020000334E8340034003427341034003401340D
:100030008634A03400340F344234403400349834D1
:10004000963480348207133403343634193403343D
:100050003A341D3400343E342234033442348207AF
:100060000A340934083406340534043402340134C3
:1000700082075334773465346534703447346534DB
:100080006E340034203456346534723431342E34B6
:100090003134653420340034533474346134723470
:1000A0007434003445346E3464340034533474345E
:1000B0006534703400344D34613472346B346534DB
:1000C00072340034533477346534653470346934B1
:1000D0006E3467340034423461346434203445343F
:1000E0006E346434003420344B3448347A34003471
:1000F000433441344C34203400348B0107309F00AA
:100100009801831698018C019F018113FB308500B3
:1001100086018312AD01AE01AF01B001B1018B22A6
:100120008B220515A522C522293084000030942396
:10013000D101D5010508D00003305005CF00501E75
:10014000272271230030B7200330B720D220031CB0
:10015000AE2834233230CB22C023A4280630B72067
:100160000930B7208323DE2071231622A228DA006B
:1001700034235A08003E2220CB22C0235A08013ED5
:100180002220D80003010E2234235A08023E2220E6
:10019000DD0010238A229C21551AD0282E21CB283D
:1001A000551208003608AD003708AE003808AF0019
:1001B0003908B0003D30840009210800D5143E30D4
:1001C000DD004D22323021213A3004214230042119
:1001D00034232930CB2205113630DD004D222D305D
:1001E000DD00E721551A01298B22453084000921C1
:1001F0000318051537213D30840009210318EB2829
:10020000F128D50105150800DD004D225D082121EA
:10021000080000083002031C2029031D2029840344
:1002200000082F02031C2029031D20298403000835
:100230002E02031C2029031D2029840300082D02FF
:10024000080084002D088000840A2E088000840A9B
:100250002F088000840A300880000800D118322955
:10026000802134293721562110238A220800D70102
:100270005D088400320880070330D30050218403D6
:100280008403330880070230D300502184033408EC
:100290008007840A031C4D29800A3508800708005E
:1002A000570D840A8007D30B5029080003305D07DF
:1002B000840003300002031C7F29031D722984037C
:1002C00093300002031C7F29031D722984038730A9
:1002D0000002031C7F29031D7229840300300002E1
:1002E000031C7F295D08840000308000840A873069
:1002F0008000840A93308000840A03308000080064
:100300009021372103305D078400801F8E298001F2
:10031000840380018403800184038001902108000C
:10032000B209B309B409B509B20F9B29B30F9B29D0
:10033000B40F9B29B50A0800CB21551ACA29050814
:10034000D000D52305085006031D9C290330500515
:10035000CE004F0603199C290310CF0D4E08CF067F
:100360004F080239D2005106D101CF18BF294E08DB
:10037000CF00DC035C189C29DC189C29C8290230BA
:10038000D1004E08CF00DC0A5C189C29DC189C299F
:100390004E08CF000800D5180B2A051AE729851D3D
:1003A000F3292030D6005510CC23051AE329851DEA
:1003B000F329D603031DD42901300E220430D600C0
:1003C0005514D511D4290130D5190B2A062A8519BF
:1003D0000B2ACC238519F129D518E929051EF32903
:1003E000E92955160B2A2030D6005510D515CC23F7
:1003F000051A052A8519052AD603031DF729FF309A
:100400000E220430D6005514F729FF3055180B2A58
:100410000E22051ECB29D5115510080058070739A3
:10042000D8002F20D9001622102308000430D30052
:10043000353084005808D7000310D70DD70D570862
:10044000012080008403D70AD30B1F2A0800D5148B
:1004500036308400043094233630DD0010238C3095
:100460004F233F30CB228A229C21051A472AB5010F
:10047000B401B3010430D01D8030B200D118412A3C
:1004800090212930DD0037213630DD00332A293034
:10049000840003019E23D5100800AD01AE01AF0119
:1004A000B001B1012030D3002908A5002A08A60018
:1004B0002B08A7002C08A8005D0884000310251C49
:1004C0007B2A0008AE07031C6A2AAF0F6A2AB00F06
:1004D0006A2AB10A840A0008AF07031C722AB00F07
:1004E000722AB10A840A0008B007031C782AB10AEC
:1004F000840A0008B107B10CB00CAF0CAE0CAD0C07
:10050000A80CA70CA60CA50C5D08D30B5D2A013026
:10051000B10008004D222D3084000008C9000830C9
:10052000C800C90C031C982A8615061506119B2ABB
:10053000861106150611C80B912A840A323004026E
:10054000031C8D2A861786130800C92303308600F2
:100550000616C9230612033086000616CC2306129F
:10056000033086000616CC230612023086000616DB
:10057000CF23061220304F2308304F2301304F2362
:1005800006304F230E304F2308000030CB220930B5
:10059000CB22BE230800DB003820FF390319D42A00
:1005A0005323DB0A5B08CC2A08002030C600A001D8
:1005B000A101A201A301A4015D0884000008A50017
:1005C000840A0008A600840A0008A700840A00081C
:1005D000A8000310A50DA60DA70DA80D031825143E
:1005E000A00DA10DA20DA30DA40DC603031DF92A94
:1005F0000800203084000523840A0523840A05238B
:10060000840A0523840A0523E92A03300007C7006A
:10061000C719800030300007C700C71B80000800E2
:10062000D52202304F2320305323230E2D232308BD
:100630002D232C305323220E2D2322082D23210E6F
:100640002D232E30532321082D23200E2D23200867
:100650002D233A30CB22302308000F39303E532B64
:10066000803059044F23080001304F2308008601D1
:10067000831608308600831206138616FF30CC00DE
:1006800006160608CB000612000000000616000041
:100690000612CC0303194E2BCB19402B0800CA00BD
:1006A000D4010613562BCA005414061737238601AB
:1006B000831600308600831286120613541806171C
:1006C000F03086054A0E0F39860406160000061221
:1006D000F03086054A080F39860406160000061217
:1006E00008003630DD008400083094233A3084005E
:1006F0000C3094233E308400103094234230840028
:100700001430942308003630840008309E233A3099
:1007100084000C309E233E30840010309E234230F3
:10072000840014309E230800F0000430D300B72367
:100730008000F00A840AD30B972B0800F0000430E5
:10074000D3000008A823840AF00AD30BA12B0800C9
:1007500083169A0070089B001C1555309D00AA3026
:100760009D009C149C18B22B1C1183120800831648
:1007700070089B001C141A0883120800C323C323AB
:10078000C323C3230800C623C6230800FF30CC00C0
:10079000D72B8030CC00D72B4030CC00D72B20304B
:1007A000CC00D72B1030CC00D72B0230CC00FF3040
:0C07B000CD00CD0BD92BCC0BD72B0800B3
:084000005700330043004400A7
:02400E00303F41
:10420000DF006500DC0017008000960098000000C9
:10421000800084001E00000020000B002000000031
:104220006400000000000000D00047001F000000F4
:00000001FF
